:02000000040AF0
:080008009F0C0200080C060029
:10001000640A170C27000000E7020B0A000000002A
:10002000000000084B0C2800F90C29000000E90230
:10003000160AE802140A000866061C0A0909660680
:100040001C0A6607210A0909090909090909090998
:1000500009090909090966071C0A090909090909A1
:1000600009096607670A0909090909096607740A7F
:10007000090966070008090909096607D70AE00A9D
:100080006606400A09096606400A6607450A090924
:100090000909090909090909090909090909660775
:1000A000400A09090909090909096607670A0909CE
:1000B000090909096607740A09096607770A09091F
:1000C00009096607D70AE00A000C2600400A010C5D
:1000D00026001209000C26001209010C2600120944
:1000E000000C26001209400A010C2600400A030CED
:1000F000260012091C09010C260012091C09030C18
:10010000260012091C09010C260012091C09030C07
:10011000260012091C09010C260012091C09030CF7
:10012000260012091C09010C260012091C09030CE7
:10013000260012091C09010C260012091C09030CD7
:10014000260012091C09010C260012091C09030CC7
:10015000260012091C0912091C0912091C0912099E
:100160001C0912091C0912091C0912091C0912098F
:100170001C0912091C0912091C0912091C0912097F
:100180001C0912091C0912091C0912091C0912096F
:100190001C09040C26001209120912091209000C8C
:1001A000260012091209120912091C09C90A020CB7
:1001B000260012091209010C260012091209400A30
:1001C000030C26001209000C26001209030C26005D
:1001D0001209000C26001209120912091209040C56
:1001E00026001209000C26001209040C2600120930
:0801F000000C26001209400A70
:021FFE00E90FE9
:00000001FF
